BL51 BANKED LINKER/LOCATER V5.03                                                        06/15/2006  17:47:46  PAGE 1


BL51 BANKED LINKER/LOCATER V5.03, INVOKED BY:
C:\KEIL\C51\BIN\BL51.EXE STARTUP.obj, main.obj, delay.obj TO UART1 RAMSIZE (256) CODE (0X0000-0X1FFF)


MEMORY MODEL: SMALL


INPUT MODULES INCLUDED:
  STARTUP.obj (?C_STARTUP)
  main.obj (MAIN)
  delay.obj (DELAY)
  C:\KEIL\C51\LIB\C51S.LIB (PRINTF)
  C:\KEIL\C51\LIB\C51S.LIB (?C?CLDPTR)
  C:\KEIL\C51\LIB\C51S.LIB (?C?CLDOPTR)
  C:\KEIL\C51\LIB\C51S.LIB (?C?CSTPTR)
  C:\KEIL\C51\LIB\C51S.LIB (?C?PLDIIDATA)
  C:\KEIL\C51\LIB\C51S.LIB (?C?CCASE)
  C:\KEIL\C51\LIB\C51S.LIB (PUTCHAR)


LINK MAP OF MODULE:  UART1 (?C_STARTUP)


            TYPE    BASE      LENGTH    RELOCATION   SEGMENT NAME
            -----------------------------------------------------

            * * * * * * *   D A T A   M E M O R Y   * * * * * * *
            REG     0000H     0008H     ABSOLUTE     "REG BANK 0"
            DATA    0008H     0014H     UNIT         _DATA_GROUP_
            DATA    001CH     0002H     UNIT         ?DT?MAIN
                    001EH     0002H                  *** GAP ***
            BIT     0020H.0   0001H.1   UNIT         _BIT_GROUP_
                    0021H.1   0000H.7                *** GAP ***
            IDATA   0022H     0001H     UNIT         ?STACK

            * * * * * * *   C O D E   M E M O R Y   * * * * * * *
            CODE    0000H     0003H     ABSOLUTE     
                    0003H     07FDH                  *** GAP ***
            CODE    0800H     035CH     UNIT         ?PR?PRINTF?PRINTF
            CODE    0B5CH     008EH     UNIT         ?C?LIB_CODE
            CODE    0BEAH     0027H     UNIT         ?PR?PUTCHAR?PUTCHAR
            CODE    0C11H     0024H     UNIT         ?CO?MAIN
            CODE    0C35H     0021H     UNIT         ?PR?MAIN?MAIN
            CODE    0C56H     0020H     UNIT         ?PR?_DELAYMS?DELAY
            CODE    0C76H     0012H     UNIT         ?PR?_DELAYUS?DELAY
            CODE    0C88H     000CH     UNIT         ?C_C51STARTUP
            CODE    0C94H     000CH     UNIT         ?PR?UARTINIT?MAIN



OVERLAY MAP OF MODULE:   UART1 (?C_STARTUP)


SEGMENT                           BIT_GROUP          DATA_GROUP 
  +--> CALLED SEGMENT          START    LENGTH     START    LENGTH
------------------------------------------------------------------
?C_C51STARTUP                  -----    -----      -----    -----
  +--> ?PR?MAIN?MAIN
BL51 BANKED LINKER/LOCATER V5.03                                                      06/15/2006  17:47:46  PAGE 2



?PR?MAIN?MAIN                  -----    -----      -----    -----
  +--> ?PR?UARTINIT?MAIN
  +--> ?CO?MAIN
  +--> ?PR?PRINTF?PRINTF
  +--> ?PR?_DELAYMS?DELAY

?PR?PRINTF?PRINTF              0020H.0  0001H.1    0008H    0014H
  +--> ?PR?PUTCHAR?PUTCHAR



SYMBOL TABLE OF MODULE:  UART1 (?C_STARTUP)

  VALUE           TYPE          NAME
  ----------------------------------

  -------         MODULE        ?C_STARTUP
  C:0C88H         SEGMENT       ?C_C51STARTUP
  I:0022H         SEGMENT       ?STACK
  C:0000H         PUBLIC        ?C_STARTUP
  D:00E0H         SYMBOL        ACC
  D:00F0H         SYMBOL        B
  D:0083H         SYMBOL        DPH
  D:0082H         SYMBOL        DPL
  N:0000H         SYMBOL        IBPSTACK
  N:0100H         SYMBOL        IBPSTACKTOP
  N:0080H         SYMBOL        IDATALEN
  C:0C8BH         SYMBOL        IDATALOOP
  N:0000H         SYMBOL        PBPSTACK
  N:0000H         SYMBOL        PBPSTACKTOP
  N:0000H         SYMBOL        PDATALEN
  N:0000H         SYMBOL        PDATASTART
  N:0000H         SYMBOL        PPAGE
  N:0000H         SYMBOL        PPAGEENABLE
  D:00A0H         SYMBOL        PPAGE_SFR
  D:0081H         SYMBOL        SP
  C:0C88H         SYMBOL        STARTUP1
  N:0000H         SYMBOL        XBPSTACK
  N:0000H         SYMBOL        XBPSTACKTOP
  N:0000H         SYMBOL        XDATALEN
  N:0000H         SYMBOL        XDATASTART
  C:0000H         LINE#         92
  C:0C88H         LINE#         99
  C:0C8AH         LINE#         100
  C:0C8BH         LINE#         101
  C:0C8CH         LINE#         102
  C:0C8EH         LINE#         151
  C:0C91H         LINE#         155
  -------         ENDMOD        ?C_STARTUP

  -------         MODULE        MAIN
  C:0000H         SYMBOL        _ICE_DUMMY_
  C:0C35H         PUBLIC        main
  D:0098H         PUBLIC        SCON
  D:0089H         PUBLIC        TMOD
  D:001CH         PUBLIC        temperature
BL51 BANKED LINKER/LOCATER V5.03                                                      06/15/2006  17:47:46  PAGE 3


  D:008DH         PUBLIC        TH1
  C:0C94H         PUBLIC        uartInit
  B:0088H.6       PUBLIC        TR1
  D:001DH         PUBLIC        humidity
  -------         PROC          UARTINIT
  C:0C94H         LINE#         42
  C:0C94H         LINE#         43
  C:0C94H         LINE#         44
  C:0C97H         LINE#         45
  C:0C9AH         LINE#         46
  C:0C9DH         LINE#         47
  C:0C9FH         LINE#         48
  -------         ENDPROC       UARTINIT
  -------         PROC          MAIN
  C:0C35H         LINE#         56
  C:0C35H         LINE#         57
  C:0C35H         LINE#         58
  C:0C38H         LINE#         59
  C:0C38H         LINE#         60
  C:0C38H         LINE#         61
  C:0C4DH         LINE#         62
  C:0C54H         LINE#         63
  -------         ENDPROC       MAIN
  -------         ENDMOD        MAIN

  -------         MODULE        DELAY
  C:0000H         SYMBOL        _ICE_DUMMY_
  D:0090H         PUBLIC        P1
  D:00B0H         PUBLIC        P3
  D:00A8H         PUBLIC        IE
  C:0C56H         PUBLIC        _DelayMs
  D:00B8H         PUBLIC        IP
  C:0C76H         PUBLIC        _DelayUs
  D:0098H         PUBLIC        SCON
  D:0088H         PUBLIC        TCON
  D:00C8H         PUBLIC        T2CON
  D:00D0H         PUBLIC        PSW
  -------         PROC          _DELAYUS
  D:0006H         SYMBOL        N
  -------         DO            
  D:0004H         SYMBOL        x
  -------         ENDDO         
  C:0C76H         LINE#         36
  C:0C76H         LINE#         37
  C:0C76H         LINE#         40
  C:0C87H         LINE#         41
  -------         ENDPROC       _DELAYUS
  -------         PROC          _DELAYMS
  D:0006H         SYMBOL        msec
  -------         DO            
  D:0004H         SYMBOL        x
  D:0002H         SYMBOL        y
  -------         ENDDO         
  C:0C56H         LINE#         54
  C:0C56H         LINE#         55
  C:0C56H         LINE#         58
  C:0C60H         LINE#         59
BL51 BANKED LINKER/LOCATER V5.03                                                      06/15/2006  17:47:46  PAGE 4


  C:0C60H         LINE#         60
  C:0C6EH         LINE#         61
  C:0C75H         LINE#         62
  -------         ENDPROC       _DELAYMS
  -------         ENDMOD        DELAY

  -------         MODULE        PRINTF
  D:0008H         PUBLIC        ?_PRINTF517?BYTE
  D:0008H         PUBLIC        ?_PRINTF?BYTE
  D:0008H         PUBLIC        ?_SPRINTF517?BYTE
  D:0008H         PUBLIC        ?_SPRINTF?BYTE
  C:0862H         PUBLIC        _PRINTF
  C:0862H         PUBLIC        _PRINTF517
  C:085CH         PUBLIC        _SPRINTF
  C:085CH         PUBLIC        _SPRINTF517
  -------         ENDMOD        PRINTF

  -------         MODULE        ?C?CLDPTR
  C:0B5CH         PUBLIC        ?C?CLDPTR
  -------         ENDMOD        ?C?CLDPTR

  -------         MODULE        ?C?CLDOPTR
  C:0B75H         PUBLIC        ?C?CLDOPTR
  -------         ENDMOD        ?C?CLDOPTR

  -------         MODULE        ?C?CSTPTR
  C:0BA2H         PUBLIC        ?C?CSTPTR
  -------         ENDMOD        ?C?CSTPTR

  -------         MODULE        ?C?PLDIIDATA
  C:0BB4H         PUBLIC        ?C?PLDIIDATA
  -------         ENDMOD        ?C?PLDIIDATA

  -------         MODULE        ?C?CCASE
  C:0BC4H         PUBLIC        ?C?CCASE
  -------         ENDMOD        ?C?CCASE

  -------         MODULE        PUTCHAR
  C:0BEAH         PUBLIC        _PUTCHAR
  -------         ENDMOD        PUTCHAR

*** WARNING L16: UNCALLED SEGMENT, IGNORED FOR OVERLAY PROCESS
    SEGMENT: ?PR?_DELAYUS?DELAY

******************************************************************************
* RESTRICTED VERSION WITH 0800H BYTE CODE SIZE LIMIT; USED: 009BH BYTE ( 7%) *
******************************************************************************

Program Size: data=32.1 xdata=0 code=1187
LINK/LOCATE RUN COMPLETE.  1 WARNING(S),  0 ERROR(S)
